:100000000C94A3000C94CB000C94CB000C94CB006C
:100010000C94CB000C94CB000C94CB000C94CB0034
:100020000C94CB000C94CB000C94CB000C94CB0024
:100030000C94CB000C94CB000C94CB000C94CB0014
:100040000C943B030C94CB000C94CB000C94CB0091
:100050000C94CB000C94CB000C94CB000C94CB00F4
:100060000C94CB000C94CB0007634236B79BD8A707
:100070001A39685618AEBAAB558C1D3CB7CC5763CD
:10008000BD6DEDFD753EF6177231BF000000803F7B
:1000900008000000BE922449123EABAAAA2ABECD97
:1000A000CCCC4C3E00000080BEABAAAAAA3E000009
:1000B0000000BF000000803F000000000008417801
:1000C000D3BB4387D1133D190E3CC3BD4282AD2B38
:1000D0003E68EC8276BED98FE1A93E4C80EFFFBE30
:1000E00001C4FF7F3F00000000000000000024006A
:1000F00027002A0000000000250028002B00000037
:10010000000023002600290004040404040404045D
:1001100002020202020203030303030301020408B2
:100120001020408001020408102001020408102061
:1001300000000008000201000003040700000000A6
:1001400000000000130711241FBECFEFD8E0DEBF70
:10015000CDBF11E0A0E0B1E0E6E6F7E102C0059016
:100160000D92A037B107D9F721E0A0E7B1E001C0B7
:100170001D92A339B207E1F710E0C3EAD0E004C052
:100180002197FE010E94AB0BC23AD107C9F70E942A
:1001900085030C94B10B0C940000833081F028F49B
:1001A000813099F08230A9F008958730A9F0883025
:1001B000C9F08430B1F4809180008F7D03C08091BC
:1001C00080008F7780938000089584B58F7784BDF9
:1001D000089584B58F7DFBCF8091B0008F77809399
:1001E000B00008958091B0008F7DF9CFCF93DF9359
:1001F000282F30E0F901E05DFE4F8491F901E45EC3
:10020000FE4FD491F901E85FFE4FC491CC23A1F0D9
:1002100081110E94CD00EC2FF0E0EE0FFF1FE250A5
:10022000FF4FA591B491EC91ED2381E090E009F4AA
:1002300080E0DF91CF91089580E090E0FACF1F93A6
:10024000CF93DF93282F30E0F901E05DFE4F8491DA
:10025000F901E45EFE4FD491F901E85FFE4FC491CD
:10026000CC23A9F0162F81110E94CD00EC2FF0E0D5
:10027000EE0FFF1FEC50FF4FA591B4918FB7F8948C
:10028000EC91111108C0D095DE23DC938FBFDF9174
:10029000CF911F910895DE2BF8CFCF93DF9390E09D
:1002A000FC01E45EFE4F2491885F9E4FFC01849127
:1002B0008823C9F090E0880F991FFC01E651FF4F99
:1002C000A591B491FC01EC50FF4FC591D4916111FF
:1002D0000DC09FB7F8948C91209582238C938881D0
:1002E000282328839FBFDF91CF910895623051F476
:1002F0009FB7F8943C91822F809583238C93E8815B
:100300002E2BEFCF8FB7F894EC912E2B2C938FBF21
:10031000EACF1F93CF93DF93182FEB0161E00E9488
:100320004D01209739F460E0812FDF91CF911F912B
:100330000C941F01CF3FD10511F461E0F5CFE12FFF
:10034000F0E0E05DFE4FE491E33031F140F4E13064
:10035000B1F0E230E1F0C038D1057CF7E4CFE7300E
:1003600029F1E83059F1E430B1F7809180008062E2
:1003700080938000D0938B00C0938A0004C084B522
:10038000806884BDC7BDDF91CF911F91089584B56A
:10039000806284BDC8BDF7CF809180008068809363
:1003A0008000D0938900C0938800EDCF8091B00089
:1003B00080688093B000C093B300E5CF8091B00017
:1003C00080628093B000C093B400DDCF8E50806413
:1003D00080937C0080917A00806480937A00809181
:1003E0007A0086FDFCCF8091780090917900089585
:1003F0004F925F926F927F928F929F92AF92BF9235
:10040000CF92DF92EF92FF92CF93DF93EC0188813E
:10041000813009F06DC0C980DA80EB80FC8028EB68
:100420003EE145E850ECC701B6010E94300B0E9446
:1004300024099B01AC018D809E80AF80B88460E070
:1004400070E080E89FE30E9438082B013C01A50181
:10045000940160E070E080E89FE30E9438089B010F
:10046000AC01C301B2010E94300BA50194010E94AE
:10047000390869877A878B879C872D853E854F85CC
:1004800058896FE672E183E89AE30E94AA08A701FF
:1004900096010E94390869837A838B839C8320E0CC
:1004A00030E040E85FE30E94650A87FD0EC080E00F
:1004B00090E0A0E8BFE389879A87AB87BC87198261
:1004C0001A821B821C8282E0888369857A858B85EB
:1004D0009C85DF91CF91FF90EF90DF90CF90BF9000
:1004E000AF909F908F907F906F905F904F90089506
:1004F000823059F7C980DA80EB80FC8028EB3EE13E
:1005000045E850ECC701B6010E94300B0E94240957
:1005100069877A878B879C8729893A894B895C8987
:100520006FE672E183E89AE30E94AA08A7019601A8
:100530000E94390869837A838B839C8320E030E0B2
:1005400040E85FE30E94650A87FDBFCF19861A86DF
:100550001B861C8619821A821B821C821882B5CFC8
:100560004F925F926F927F928F929F92AF92BF92C3
:10057000CF92DF92EF92FF92CF93DF936B017C01DA
:1005800020E030E0A9010E94A50887FD69C020E0B5
:1005900030E040E85FE3C701B6010E94650A181623
:1005A0000CF462C020E030E040E052E4C701B60144
:1005B0000E94300B4B015C010E945609EB01603236
:1005C000710514F0CFE1D0E0FE01EE0FFF1FE25DF8
:1005D000FE4F6081718190E080E00E948C090E9452
:1005E000B40A6B017C01FE01EE0FFF1FE05DFE4FC0
:1005F0006081718190E080E00E948C090E94B40AC1
:100600002B013C01BE01DD0F880B990B0E948E0966
:100610009B01AC01C501B4010E9438084B015C018B
:10062000A7019601C301B2010E9438089B01AC01E9
:10063000C501B4010E94300BA70196010E94390840
:10064000DF91CF91FF90EF90DF90CF90BF90AF9070
:100650009F908F907F906F905F904F900C942409A3
:10066000C12CD12C76019ECFC12CD12C20E8E22EBA
:100670002FE3F22E97CF1F920F920FB60F921124F5
:100680002F933F938F939F93AF93BF9380918F014D
:1006900090919001A0919101B091920130918E01C1
:1006A00023E0230F2D3758F50196A11DB11D20938E
:1006B0008E0180938F0190939001A0939101B0934C
:1006C000920180918A0190918B01A0918C01B0914F
:1006D0008D010196A11DB11D80938A0190938B011C
:1006E000A0938C01B0938D01BF91AF919F918F9199
:1006F0003F912F910F900FBE0F901F90189526E8F5
:10070000230F0296A11DB11DD2CFCF93DF93CDB79A
:10071000DEB760970FB6F894DEBF0FBECDBF7894FA
:1007200084B5826084BD84B5816084BD85B58260F6
:1007300085BD85B5816085BD80916E0081608093A7
:100740006E00109281008091810082608093810010
:100750008091810081608093810080918000816020
:10076000809380008091B10084608093B10080917B
:10077000B00081608093B00080917A0084608093A3
:100780007A0080917A00826080937A0080917A006A
:10079000816080937A0080917A00806880937A00EB
:1007A0001092C10062E084E00E944D0160E081E1AE
:1007B0000E944D0160E08AE00E944D0161E083E00B
:1007C0000E944D0161E089E00E944D0161E08BE0F3
:1007D0000E944D0183E28093B00081E08093B100DC
:1007E00082E88093800089E1809381008FEF90E020
:1007F000909387008093860000E010E08FB7F89414
:1008000080908F0190909001A0909101B090920102
:100810008FBF8092860190928701A0928801B0924A
:1008200089018EE00E94E601BC01990F880B990BAB
:100830000E948E0920E030EC4FE754E40E94AA08A1
:100840002B013C018FE00E94E601BC01990F880B4F
:10085000990B0E948E0920E030EC4FE754E40E948F
:10086000AA086B017C0180E10E94E601BC01990F9E
:10087000880B990B0E948E0920E030EC4FE754E47E
:100880000E94AA0869837A838B839C83C301B20187
:100890000E94B0029B01AC016AE077ED83E292E432
:1008A0000E94AA086D877E878F87988BC701B60143
:1008B0000E94B0029B01AC016AE077ED83E292E412
:1008C0000E94AA0869877A878B879C8720E030E09E
:1008D000A901C301B2010E94A50887FD86C220E0DC
:1008E00030E040E85FE3C301B2010E94650A1816D8
:1008F0000CF47FC2A301920160E070E080E89FE306
:100900000E9438082AE939E949E15FE30E94300B87
:100910002DEC3CEC4CE45EE30E94390829813A81DD
:100920004B815C810E94300B6D837E838F8398871F
:1009300020E030E0A901C701B6010E94A50887FDAB
:100940005FC220E030E040E85FE3C701B6010E94EB
:10095000650A18160CF458C2A701960160E070E011
:1009600080E89FE30E9438082AE939E949E15FE31A
:100970000E94300B2DEC3CEC4CE45EE30E94390805
:1009800029813A814B815C810E94300B2B013C0113
:1009900084E00E94F60010928401109285019091EB
:1009A0008301891751F08093830180927E01909298
:1009B0007F01A0928001B092810180917E0190918F
:1009C0007F01A0918001B0918101A5019401281BB4
:1009D000390B4A0B5B0BDA01C90140917A01509146
:1009E0007B0160917C0170917D01481759076A076E
:1009F0007B07B0F49091820180918301981781F078
:100A000080938201911103C021E0813009F020E040
:100A100020938401913009F4811190E09093850135
:100A200081E10E94F60020917701211103C091E03D
:100A3000813009F090E090937801213011F491E039
:100A4000811190E090937901809377018AE00E9470
:100A5000F60020917401211103C091E0813009F06A
:100A600090E090937501213019F431E039838111C0
:100A700019824981409376018093740180918501A8
:100A8000811105C080917901882309F4A2C00E94D8
:100A90007D074B015C010E947D0720ED37E040E0BF
:100AA00050E00E94D507685E7340810991090E9459
:100AB0008E0920E030E04AE754E40E94AA08A3012E
:100AC00092010E94300B20E030E040E85FE30E949A
:100AD000390829853A854B855C850E94300B6B016E
:100AE0007C01C501B40120ED37E040E050E00E94F8
:100AF000D507685E7340810991090E948E0920E044
:100B000030E04AE754E40E94AA082D813E814F81DB
:100B100058850E94300B20E030E040E85FE30E94FF
:100B200039082D853E854F8558890E94300B4B0131
:100B30005C0120E030E0A9010E94650A181644F02B
:100B40003FE6832E32E1932E33E8A32E3AE3B32E11
:100B50008092220190922301A0922401B09225015B
:100B600020E030E0A901C701B6010E94650A18160D
:100B700044F02FE6C22E22E1D22E23E8E22E2AE311
:100B8000F22EC0922601D0922701E0922801F09225
:100B9000290180911501823009F03DC180911E012B
:100BA00090911F01A0912001B091210180931A0121
:100BB00090931B01A0931C01B0931D0151E0509331
:100BC000150110921601109217011092180110923F
:100BD00019018981882309F4A2C00E947D076B0155
:100BE0007C010E947D0720ED37E040E050E00E944C
:100BF000D507685E7340810991090E948E0920E043
:100C000030E04AE754E40E94AA08A30192010E943E
:100C1000300B20E030E040E85FE30E94390829858E
:100C20003A854B855C850E94300B4B015C01C70106
:100C3000B60120ED37E040E050E00E94D507685E45
:100C40007340810991090E948E0920E030E04AE753
:100C500054E40E94AA082D813E814F8158850E944C
:100C6000300B20E030E040E85FE30E9439082D853A
:100C70003E854F8558890E94300B6B017C0120E036
:100C800030E0A9010E94650A181644F09FE6C92EBB
:100C900092E1D92E93E8E92E9AE3F92EC0920D0144
:100CA000D0920E01E0920F01F092100120E030E0AE
:100CB000A901C501B4010E94650A181644F08FE627
:100CC000882E82E1982E83E8A82E8AE3B82E80929F
:100CD000110190921201A0921301B092140180911F
:100CE0000001823009F09BC08091090190910A01B6
:100CF000A0910B01B0910C01809305019093060126
:100D0000A0930701B093080191E090930001109225
:100D100001011092020110920301109204018091CE
:100D2000860190918701A0918801B091890140913D
:100D3000700150917101609172017091730184177B
:100D40009507A607B70709F449C0809370019093EF
:100D50007101A0937201B093730185E191E00E944B
:100D6000F80180E091E00E94F80120E030E04FE7D8
:100D700053E460911E0170911F01809120019091B8
:100D800021010E94300B0E94560989E00E948901CE
:100D900020E030E040E253E460911E0170911F01B9
:100DA00080912001909121010E94300B0E945609F0
:100DB00083E00E94890120E030E04FE753E4609136
:100DC000090170910A0180910B0190910C010E9420
:100DD000300B0E9456098BE00E9489010115110514
:100DE00009F40CCD0E94000009CD412C512C320198
:100DF00081CD412C512C50E8652E5FE3752E7ACDC4
:100E0000C12CD12C7601A8CDC12CD12C40E8E42EE8
:100E10004FE3F42EA1CD80E090E0DC01C7CE80E06E
:100E200090E0DC0169CFEAE7F1E082E390E0A0E046
:100E3000B0E080839183A283B383148215821682EB
:100E4000178281E08087818712861386E7E7F1E0C9
:100E5000808311821282E4E7F1E0808311821282A2
:100E600008958F929F92AF92BF92CF92DF92EF92AE
:100E7000FF92CF93DF93EC01688179818A819B8116
:100E8000611571058105910521F464E279ED8BE529
:100E900097E02DE133EF41E050E00E94D507490192
:100EA0005A019B01AC01A7EAB1E40E94F4076B016F
:100EB0007C01ACEEB4EFA50194010E940208C60EBD
:100EC000D71EE81EF91EF7FE06C081E0C81AD10839
:100ED000E10880E8F80AC882D982EA82FB82C70169
:100EE000B6019F77DF91CF91FF90EF90DF90CF9089
:100EF000BF90AF909F908F9008958F929F92AF92E6
:100F0000BF92CF92DF92EF92FF9260912A0170918F
:100F10002B0180912C0190912D01611571058105A6
:100F2000910521F464E279ED8BE597E02DE133EF53
:100F300041E050E00E94D50749015A019B01AC01F4
:100F4000A7EAB1E40E94F4076B017C01ACEEB4EFB8
:100F5000A50194010E940208C60ED71EE81EF91EC4
:100F6000F7FE06C081E0C81AD108E10880E8F80A57
:100F7000C0922A01D0922B01E0922C01F0922D0117
:100F8000C701B6019F77FF90EF90DF90CF90BF90A1
:100F9000AF909F908F90089560932A0170932B01DA
:100FA00080932C0190932D010895052E97FB1EF43C
:100FB00000940E94EC0757FD07D00E94070807FC29
:100FC00003D04EF40C94EC07509540953095219544
:100FD0003F4F4F4F5F4F0895909580957095619565
:100FE0007F4F8F4F9F4F08950E942908A59F900D16
:100FF000B49F900DA49F800D911D11240895B7FFFB
:101000000C94F4070E94F407821B930B0895A1E24D
:101010001A2EAA1BBB1BFD010DC0AA1FBB1FEE1F72
:10102000FF1FA217B307E407F50720F0A21BB30BBD
:10103000E40BF50B661F771F881F991F1A9469F739
:1010400060957095809590959B01AC01BD01CF0195
:101050000895A29FB001B39FC001A39F700D811D91
:101060001124911DB29F700D811D1124911D0895B1
:101070005058BB27AA270E9450080C942B0A0E94A4
:101080001D0A38F00E94240A20F039F49F3F19F419
:1010900026F40C94F3090EF4E095E7FB0C94ED09AB
:1010A000E92F0E943C0A58F3BA17620773078407B6
:1010B000950720F079F4A6F50C945E0A0EF4E095FD
:1010C0000B2EBA2FA02D0B01B90190010C01CA0102
:1010D000A0011124FF27591B99F0593F50F4503EAD
:1010E00068F11A16F040A22F232F342F4427585F9F
:1010F000F3CF469537952795A795F0405395C9F7B7
:101100007EF41F16BA0B620B730B840BBAF091506E
:10111000A1F0FF0FBB1F661F771F881FC2F70EC00D
:10112000BA0F621F731F841F48F4879577956795E0
:10113000B795F7959E3F08F0B0CF9395880F08F0CC
:101140009927EE0F9795879508950E94C90908F48D
:1011500081E008950E94BE080C942B0A0E94240A84
:1011600058F00E941D0A40F029F45F3F29F00C94CA
:10117000ED0951110C945F0A0C94F3090E943C0A8A
:1011800068F39923B1F3552391F3951B550BBB27B6
:10119000AA2762177307840738F09F5F5F4F220FFB
:1011A000331F441FAA1FA9F335D00E2E3AF0E0E8F2
:1011B00032D091505040E695001CCAF72BD0FE2F3C
:1011C00029D0660F771F881FBB1F261737074807D0
:1011D000AB07B0E809F0BB0B802DBF01FF27935888
:1011E0005F4F3AF09E3F510578F00C94ED090C9456
:1011F0005F0A5F3FE4F3983ED4F386957795679551
:10120000B795F7959F5FC9F7880F911D96958795BC
:1012100097F90895E1E0660F771F881FBB1F6217DB
:1012200073078407BA0720F0621B730B840BBA0B99
:10123000EE1F88F7E095089529F416F00C94ED0957
:101240000C945E0A0C94F3090E94440AA8F39638A1
:10125000A0F707F80F92E8942BE33AEA48EB5FE730
:101260000E94460B0F920F920F924DB75EB70F92EE
:101270000E94FC0AE8E6F0E00E94F6094F915F91B7
:10128000EF91FF91E595EE1FFF1F49F0FE57E068D3
:101290004427EE0F441FFA95E1F74195550B0E9444
:1012A000760A0F9007FE0C946A0A08950E945D0961
:1012B0006894B1110C945F0A08950E94440A88F062
:1012C0009F5798F0B92F9927B751B0F0E1F0660F0A
:1012D000771F881F991F1AF0BA95C9F714C0B1304B
:1012E00091F00E945E0AB1E008950C945E0A672FA7
:1012F000782F8827B85F39F0B93FCCF3869577957A
:101300006795B395D9F73EF4909580957095619562
:101310007F4F8F4F9F4F0895E89409C097FB3EF48D
:1013200090958095709561957F4F8F4F9F4F992332
:10133000A9F0F92F96E9BB279395F69587957795B0
:101340006795B795F111F8CFFAF4BB0F11F460FF70
:101350001BC06F5F7F4F8F4F9F4F16C0882311F0C8
:1013600096E911C0772321F09EE8872F762F05C0DC
:10137000662371F096E8862F70E060E02AF09A9577
:10138000660F771F881FDAF7880F9695879597F96C
:101390000895990F0008550FAA0BE0E8FEEF161606
:1013A0001706E807F907C0F012161306E407F50759
:1013B00098F0621B730B840B950B39F40A2661F0CD
:1013C000232B242B252B21F408950A2609F4A14070
:1013D000A6958FEF811D811D089597F99F6780E87D
:1013E00070E060E008959FEF80EC0895DF93CF9365
:1013F0001F930F93FF92EF92DF927B018C01689411
:1014000006C0DA2EEF010E94430BFE01E894A5917D
:101410002591359145915591A6F3EF010E94500811
:10142000FE019701A801DA9469F7DF90EF90FF9031
:101430000F911F91CF91DF91089500240A94161601
:10144000170618060906089500240A9412161306B2
:10145000140605060895092E0394000C11F4882340
:1014600052F0BB0F40F4BF2B11F460FF04C06F5F5C
:101470007F4F8F4F9F4F089557FD9058440F551F32
:1014800059F05F3F71F04795880F97FB991F61F006
:101490009F3F79F087950895121613061406551F7D
:1014A000F2CF4695F1DF08C0161617061806991FE9
:1014B000F1CF86957105610508940895E894BB27DE
:1014C00066277727CB0197F908950E94C90908F488
:1014D0008FEF08959B01AC0160E070E080E89FE32E
:1014E0000C94AA080C94ED090C949D0B0E94440ADC
:1014F000D8F39923C9F3940F511DA3F39150504091
:1015000094F059F0882332F0660F771F881F9150AE
:101510005040C1F79E3F51052CF7880F911D9695BD
:10152000879597F908955F3FACF0983E9CF0BB27F4
:10153000869577956795B79508F4B1609395C1F74F
:10154000BB0F58F711F460FFE8CF6F5F7F4F8F4FED
:101550009F4FE3CF0C945F0A16F00C949D0B0C94F4
:10156000F30968940C94ED090E94440AA8F39923A6
:10157000C1F3AEF3DF93CF931F930F93FF92C92F65
:10158000DD2788232AF02197660F771F881FDAF757
:1015900020E030E040E85FEB9FE3883920F0803EB8
:1015A00038F021968F770E943908E0E9F0E004C016
:1015B0000E943908EDEBF0E00E94F6098B01BE01B4
:1015C000EC01FB2E6F5771097595771F880B990BEE
:1015D0000E948E0928E132E741E35FE30E94430B5A
:1015E000AF2D9801AE01FF900F911F91CF91DF9128
:1015F0000E9450080C942B0AFA01DC01AA0FBB1FB1
:101600009B01AC01BF5728F4222733274427507889
:1016100020C0B75190F4AB2F0024469537952795FD
:10162000011CA395D2F3002071F0220F331F441F39
:10163000B395DAF30ED00C94380861307105A0E848
:101640008A07B94630F49B01AC01662777278827C3
:101650009078309621F0208331834283538308951C
:101660000E94430B0C942B0A0E941D0A38F00E9422
:10167000240A20F0952311F00C94ED090C94F30941
:1016800011240C945F0A0E943C0A70F3959FC1F3E9
:10169000950F50E0551F629FF001729FBB27F00D20
:1016A000B11D639FAA27F00DB11DAA1F649F662775
:1016B000B00DA11D661F829F2227B00DA11D621FC4
:1016C000739FB00DA11D621F839FA00D611D221F7E
:1016D000749F3327A00D611D231F849F600D211D62
:1016E000822F762F6A2F11249F5750409AF0F1F0E5
:1016F00088234AF0EE0FFF1FBB1F661F771F881F4E
:1017000091505040A9F79E3F510580F00C94ED098F
:101710000C945F0A5F3FE4F3983ED4F38695779587
:101720006795B795F795E7959F5FC1F7FE2B880FF3
:10173000911D9695879597F908959F3F31F09150A7
:1017400020F4879577956795B795880F911D9695A5
:10175000879597F90895EE0FFF1F0590F491E02DFE
:061760000994F894FFCF8C
:1017660000000000000000000000000000CDCCCC0E
:101776003D0000003F0000000000000000000000E7
:101786000000CDCCCC3D0000003F0100000000046D
:101796006B03EC027F022102D2018D01530121016C
:1017A600F600D200B300980081006E005D004F0085
:1017B600430038002F00280021001B0017001200EC
:1017C6000F000C00090007000500040002000100DC
:00000001FF
